:020000040800F2
:10000000600900204501000819110008811000084E
:1000100015110008B1010008FB2F000800000000C6
:10002000000000000000000000000000BD260008E5
:10003000110E0008000000005D22000809290008D8
:100040005F0100085F0100085F0100085F01000810
:100050005F0100085F0100085F0100085F01000800
:100060005F0100085F0100085F0100085F010008F0
:100070005F0100085F0100085F0100085F010008E0
:100080005F0100085F0100085F0100085F010008D0
:100090005F0100085F0100085F0100085F010008C0
:1000A0005F0100085F0100085F0100085F010008B0
:1000B0005F010008712900085F0100085F01000866
:1000C0005F0100085F0100085F0100085F01000890
:1000D0005F010008512B0008AD2B0008912C00088F
:1000E0005F0100085F0100085F0100085F01000870
:1000F0005F0100085F0100085F0100085F01000860
:100100005F0100085F0100085F0100085F0100084F
:100110005F0100085F0100085F0100085F0100083F
:100120005F0100085F0100085F0100085F0100082F
:10013000DFF80CD000F02AF8004800470131000831
:10014000600900200648804706480047FEE7FEE7B2
:10015000FEE7FEE7FEE7FEE7FEE7FEE7FEE7FEE777
:100160000D29000831010008D2B201E000F8012B8E
:10017000491EFBD270470022F6E710B513460A4627
:1001800004461946FFF7F0FF204610BD064C074D08
:1001900006E0E06840F0010394E807009847103457
:1001A000AC42F6D3FFF7C8FF84340008A43400083B
:1001B00000BFFEE710B502460B460020002104E018
:1001C000545C0444E0B24C1CE1B29942F8DBC443F5
:1001D000E0B2441CE0B210BDFEB5002000900190DA
:1001E000029000F067FF3A4800780A2822D1394887
:1001F000007839490978884218D13648407836491C
:100200004978884212D13348007A3349097A8842C2
:100210000CD13048407A3049497A884206D12F487B
:10022000008840F400402D49088003E0142129484B
:10023000FFF7A1FF2948008800F40040002846D0BD
:10024000274800210160017126480160017126489C
:100250000160017125480160017100202149087089
:100260001C48007948701B4840798870194880798B
:10027000C8701848C079087100201D4908701948D5
:10028000407848701748807888701648C078C870E1
:1002900014480079087113484078040611488078A2
:1002A00005041048C0780602601930440D490979E8
:1002B000471801200F49087000F0FCFE0020044997
:1002C00008700649088014210248FFF754FFFEBD5C
:1002D00009000020D40100200C0000200A000020AA
:1002E00034000020160000203C00002041000020C7
:1002F0001B0000204900002010B588B07F4800781E
:10030000012838D100207D490870FC207C49087004
:10031000112048707B48007888707A484078C8700F
:100320007848807808717748C078487175480079B6
:10033000887107217248FFF73DFF7149C87100209D
:1003400071490860FF22E121012001F0D5FE082358
:100350006B4AA821012001F091FE012001F0C8F9AB
:1003600001206A49C1F8A40169490870002069495F
:10037000088000F09FFE6748008840F6B831884248
:100380007BDC00F097FE604884380068002857D175
:1003900000F090FE6946012001F04EFE0446204622
:1003A00002F0DAF95CA002F0E1F904F04000402824
:1003B000EDD100208DF80A000721684600F029FDE4
:1003C00055A002F0D3F99DF801004E490978884202
:1003D00054D19DF802004B49497888424ED19DF88E
:1003E000030048498978884248D19DF8040045496E
:1003F000C978884242D19DF805004249097988426E
:100400003CD14348007801281BD141480078401C6A
:100410003F49087012203A49487007213848FFF7D1
:10042000C9FE3749C8710020374908600823344A9B
:10043000A821012001F022FE01203449C1F8A401C5
:1004400058E00020324908700E21344800F0E1FCE9
:1004500031A002F08BF932480178012001F0A2F9B5
:1004600010202E4948700E212C4802F069F92DA069
:1004700002F07CF9012008B010BD16E000202249EE
:10048000086011201E49487007211D48FFF792FEA1
:100490001B49C87108230A46A821012001F0EEFD7E
:1004A00001201A49C1F8A40124E000201549087070
:1004B00048708870C87008711B490870487088704F
:1004C000C87008711949087048708870C870087140
:1004D0001749087048708870C870087130200F493B
:1004E00048700E210D4802F02BF912A002F03EF9DF
:1004F0000120C0E700F0DEFD0020BCE74600002040
:100500004A00002034000020A481214200802142C2
:100510008A000020260000200A000000C8030020F6
:10052000320000204F4B0A00410000201B00002039
:1005300016000020333030300A00000010B588B0BB
:100540005648008840F6B831884271DA544800684D
:1005500000286ED100F0AEFD6946012001F06CFD6F
:10056000044604F040004028F3D100208DF80A0032
:100570009DF8010078B99DF8020060B99DF803006C
:1005800048B900204749087048708870C8700871E1
:10059000012008B010BD44480078072803D0424825
:1005A00000780D280FD100203E4908709DF800000A
:1005B00048709DF8010088709DF80200C8709DF891
:1005C0000300087159E038480078082810D19DF8D8
:1005D0000100344908709DF8020048709DF803003E
:1005E00088709DF80400C8709DF80500087144E00B
:1005F0002D480078092803D02B4800780E2819D1FF
:100600000020284908709DF8010080F053004870D0
:100610009DF8020080F0430088709DF8030080F090
:100620004400C8709DF8040080F05800087124E070
:1006300028E024E01C48007814280FD10020194934
:1006400008709DF8040048709DF8050088709DF8BA
:100650000600C8709DF8070008710EE000201149DF
:1006600008709DF8010048709DF8020088709DF8A0
:100670000300C8709DF804000871012089E700F0AC
:1006800019FD08E000200749087048708870C8709C
:10069000087101207DE700207BE700003A00002080
:1006A00020812142410000203200002010B500F0DE
:1006B00001FDFE480078082829D1FD4800787528FA
:1006C00025D1FB484078702821D1F94880786428EA
:1006D0001DD1F748C078612819D1F54800797428F0
:1006E00015D1F3484079652811D10020EF490870F1
:1006F00000BFF048006800F4E060EF490843001DC7
:10070000EC490860BFF34F8F00BF00BFFEE7E84829
:100710000078752807D0E6480078FA2803D0002032
:10072000E249087010BDE14800780E2800DAF9E7C8
:10073000DE480078401EDE49085CFB2800D0F1E767
:10074000DB48807AA02804D1D8480078152800D04A
:10075000E8E7D64800780E281ED1D5480078FA2858
:1007600014D1D348407BFB2810D1D448008840F4F2
:100770000040D24908800020CC4908700E21CC48A6
:1007800000F047FBCEA001F0F1FF4AE00020C7498E
:100790000870CA49088044E0C448007815281ED172
:1007A000C3480078FA2814D1C148007DFB2810D135
:1007B000C248008840F40040C04908800020BB497E
:1007C00008701521BA4800F024FBBDA001F0CEFF4F
:1007D00027E00020B5490870B849088021E0B348F7
:1007E000007811281DD1B2480078FA2814D1B048F9
:1007F000007CFB2810D1B148008840F40040AF498C
:1008000008800020A94908701121A94800F001FBC7
:10081000ABA001F0ABFF04E00020A4490870A74999
:100820000880A648008800F40040002871D000F03D
:1008300041FC9F488079A34988719D48C179A148AE
:10084000C1719B48017A9F4801729948417A9D483D
:1008500041729748807A9B498872084680799A4904
:1008600088719848C1799848C1719648017A96482C
:1008700001729448417A944841729248807A94284F
:100880004CD018DC732834D00CDC252825D004DCAF
:1008900021281AD022287DD11BE0262821D07128BA
:1008A000F9D122E0742828D075282AD078282CD0B5
:1008B0008228F0D12EE0A03809286BD2DFE800F0C2
:1008C000329CA0F5F4F3F2F1F00000207D4988722B
:1008D000DAE100207B498872D6E1002079498872EC
:1008E000D2E1002077498872CEE1002075498872F4
:1008F000CAE1002073498872C6E1002071498872FC
:10090000C2E100206F498872BEE100206D49887203
:10091000BAE1BDE100206B498872B5E10020694968
:100920008872B1E1002061490870664880796749A2
:1009300088716448C1796548C1716248017A634829
:1009400001726048417A614841725E48807A5F492D
:1009500088725748407B5B4948735548817B5948AA
:1009600081735348C17B5748C1735148017C554836
:1009700001744F48417C534841744D48407B544971
:1009800008704B48807B48704948C07B8870484855
:10099000007C00E077E1C8704548407C0871012088
:1009A0004C49087000204C490880012000F0A0FE4E
:1009B0004AA001F0DBFE04E0FFF79EFC044604B110
:1009C00000E0F9E700BF45A001F0D0FE0020454956
:1009D000087048708870C870087143490870487082
:1009E0008870C87008714149087048708870C87074
:1009F00008713449887247E100203249887243E126
:100A00003B48007830B9384800210160017101206D
:100A1000374908703448407848B93348807830B94D
:100A20003148C07818B93048007900B92CE100206D
:100A30001E490870234880792E4988712148C17960
:100A40002C48C1711F48017A2A4801721D48417A19
:100A5000284841721B48807A264988720120C87252
:100A600006200873002048731F48017821488173CD
:100A70001D4841781F48C1731B4881781D48017487
:100A80001948C1781B484174174801791948817485
:100A9000162101F055FE322002F0DEFA16212BE07D
:100AA000A8E0ECE0E7E0E2E03AE038E00300002014
:100AB0000C0100200CED00E00000FA05040000200D
:100AC0000A000000000300209C020020C803002050
:100AD0003400002046000020260000203030303056
:100AE0000A000000410000201B000020160000202A
:100AF0002B00002064030020664800F08AF9AFF262
:100B0000400001F033FE002063490870487088708F
:100B1000C87008716149087061498872B4E0B3E037
:100B200000206049087060480178012000F03AFE1A
:100B300000205E4908805EA001F018FE04E0FFF787
:100B4000FDFC044604B100E0F9E700BF58A001F045
:100B50000DFE534880794F4988715148C1794D48FD
:100B6000C1714F48017A4B4801724D48417A49485A
:100B700041724B48807A474988720120C87206202A
:100B80000873002048734C480178424881734A48F2
:100B900041784048C173484881783E4801744648CE
:100BA000C1783C484174444801793A48817416211F
:100BB00001F0C6FD322002F04FFA1621354800F050
:100BC00028F93CA001F0D2FD00203B490870487094
:100BD0008870C87008713049087048708870C87093
:100BE00008713649087048708870C87008712C49BF
:100BF000887249E03248407B2B4908702848807948
:100C0000304988712648C1792E48C1712448017A3B
:100C10002C4801722248417A2A4841722048807A41
:100C200028498872012048700E21264801F088FD6D
:100C3000322002F011FA1C4800782349088001F0A4
:100C400047FD00201C49087048708870C870087102
:100C50001149087048708870C87008711749087089
:100C600048708870C87008710D4988720CE00020C7
:100C70000B49887208E000200949887204E00020CE
:100C80000749887200E000BF00BF00200F490880BC
:100C900000BF47E5640300201B0000202B0000205C
:100CA0000003002003000020320000203A00002052
:100CB000343434340A0000004100002016000020C3
:100CC0000C0100202C04002034050020040000202A
:100CD000FA204A49087010204870002088700021CE
:100CE0004648C1700171417100204449887100215A
:100CF0004248C1710172417200204049C87400210C
:100D00003E480175FB203D494875FA203C49087072
:100D1000102048700020887000213948C17001718E
:100D2000417100203649887100213548C171017236
:100D300041720020324981F84B000021304880F890
:100D40004C10FB202E4981F84D00FA202D490870E7
:100D5000102048700020887000212A48C17001715D
:100D6000417100202749887100212648C171017214
:100D7000417200202349C872002122480173FB20E0
:100D800020494873FA20204908701020487000203C
:100D9000887000211C48C1700171417100201A49FE
:100DA000887100211848C1710172417200201649F2
:100DB000C874002114480175FB2013494875FA20B6
:100DC00012490870102048700020887000210F48D8
:100DD000C1700171417100200C49887100210B48DC
:100DE000C1710172417200200849C8720021074890
:100DF0000173FB2005494873704700009C020020E6
:100E0000000300202C04002064030020C8030020FD
:100E100070472DE9F04104460E460DE02578281173
:100E200000F030F9074601F097FC284600F02AF957
:100E3000074601F091FC641C301EA6F10101CEB200
:100E4000ECD1BDE8F081000030B5044604254FF434
:100E5000302000F06FF80546042D17D10C480069CA
:100E600040F002000A49086108464461006940F008
:100E7000400008614FF4302000F05CF8054604485B
:100E8000006941F6FD71084001490861284630BDFE
:100E90000020024004200B49C96801F0010109B19A
:100EA00001200EE00749C96801F0040109B10220E0
:100EB00007E00449C96801F0100109B1032000E00E
:100EC00004207047002002400348006940F0800081
:100ED00001490861704700000020024070B50446D7
:100EE0000D460426F00200F025F80646042E11D126
:100EF0000948006940F00100074908612580F002B7
:100F000000F018F806460448006941F6FE710840F2
:100F100001490861304670BD002002400248034983
:100F2000486003484860704723016745002002403D
:100F3000AB89EFCD00B502460423FFF7ABFF0346B4
:100F400003E0FFF7A7FF0346521E012B01D1002A41
:100F5000F7D102B90523184600BD2DE9F04102463C
:100F600000250026002000230024002791F803C05C
:100F70000CF00F0591F803C00CF0100CBCF1000F41
:100F800003D091F802C04CEA050591F800C0BCF10D
:100F9000000F31D0146800202BE04FF0010C0CFA48
:100FA00000F3B1F800C00CEA03069E4220D1830092
:100FB0004FF00F0C0CFA03F7BC4305FA03FC4CEAA4
:100FC000040491F803C0BCF1280F06D14FF0010CC6
:100FD0000CFA00FCC2F814C00AE091F803C0BCF19E
:100FE000480F05D14FF0010C0CFA00FCC2F810C0FC
:100FF000401C0828D1D31460B1F800C0BCF1FF0F29
:1010000034DD546800202EE000F1080C4FF0010898
:1010100008FA0CF3B1F800C00CEA03069E4221D195
:1010200083004FF00F0C0CFA03F7BC4305FA03FCE6
:101030004CEA040491F803C0BCF1280F05D100F17B
:10104000080C08FA0CF8C2F8148091F803C0BCF13F
:10105000480F07D100F1080C4FF0010808FA0CF80E
:10106000C2F81080401C0828CED35460BDE8F0813F
:10107000416170470161704701460A8890B270472C
:1010800000BFFEE70146002001F00F02092A04DC40
:1010900001F00F0202F1300003E001F00F023732DD
:1010A000D0B270474CF6CC40014908607047000050
:1010B0000030004010B500F013F810BD70B50546C3
:1010C0000C4645F2555000F01FF8284600F010F885
:1010D000204600F013F800F003F8FFF7E3FF70BDBF
:1010E0004AF6AA200149086070470000003000401D
:1010F00001494860704700000030004001498860A5
:10110000704700000030004001490860704700004F
:101110000030004000BFFEE7704700007CB5054688
:1011200012A103C9CDE900010821284601F09EFA69
:1011300005236A463021284600F0A0FF05236A46B1
:101140001021284600F00AFF002406E01DF80400E4
:10115000A52800D003E0601CC4B2052CF6DB00BF5C
:10116000052C01D001207CBD0020FCE7A5A5A5A58C
:10117000A500000008B501211C2001F081F84020E5
:10118000ADF8000010208DF8030003208DF8020058
:1011900069463248FFF7E1FE40213048FFF76AFF19
:1011A0001020ADF8000069462D48FFF7D6FE10214B
:1011B0002B48FFF75FFF8020ADF8000048208DF836
:1011C000030003208DF8020069462448FFF7C5FE9E
:1011D0004FF40070ADF8000010208DF803000320DC
:1011E0008DF8020069461D48FFF7B7FE4FF4007105
:1011F0001A48FFF73FFF4FF48050ADF800006946F2
:101200001648FFF7AAFE4FF480511448FFF732FF4B
:101210004FF48070ADF8000048208DF803000320E3
:101220008DF8020069460D48FFF797FE01F04CF972
:1012300001F008F900200B49086001200A49C1F8B3
:101240009001002007490C31086001200749C1F8CE
:10125000B0010821002001F009FA08BD000C01408E
:101260000008014098812142000021420080214273
:1012700010B5044602222321204600F03DFF05233D
:101280001E4A2A21204600F0F9FE05231B4A302180
:10129000204600F0F3FE3F222121204600F02CFFE3
:1012A00001222221204600F027FF1A222521204674
:1012B00000F022FF24222621204600F01DFF0F22ED
:1012C0002021204600F018FF0A223121204600F09C
:1012D00013FF01223D21204600F00EFF00223C2199
:1012E000204600F009FF70222721204600F004FF6D
:1012F000FF22E221204600F0FFFE10BD313400083D
:1013000010B5044602222321204600F0F5FE0423F6
:101310001E4A2A21204600F0B1FE04231B4A302138
:10132000204600F0ABFE30222121204600F0E4FEF2
:1013300001222221204600F0DFFE12222521204634
:1013400000F0DAFE24222621204600F0D5FE0F22EE
:101350002021204600F0D0FE08223121204600F056
:10136000CBFE01223D21204600F0C6FE00223C219A
:10137000204600F0C1FE70222721204600F0BCFE6E
:10138000FF22E221204600F0B7FE10BD68340008BD
:1013900010B5044602222321204600F0ADFE0423AE
:1013A0001E4A2A21204600F069FE04231B4A3021F0
:1013B000204600F063FE30222121204600F09CFEF2
:1013C00001222221204600F097FE282225212046D6
:1013D00000F092FE0C222621204600F08DFE0F2206
:1013E0002021204600F088FE06223121204600F010
:1013F00083FE01223D21204600F07EFE00223C219A
:10140000204600F079FE70222721204600F074FE6D
:10141000FF22E221204600F06FFE10BD5E3400087E
:1014200010B5044602222321204600F065FE042365
:101430001E4A2A21204600F021FE04231B4A3021A7
:10144000204600F01BFE30222121204600F054FEF1
:1014500001222221204600F04FFE1622252120469F
:1014600000F04AFE04222621204600F045FE0F220D
:101470002021204600F040FE08223121204600F0C5
:101480003BFE01223D21204600F036FE00223C2199
:10149000204600F031FE70222721204600F02CFE6D
:1014A000FF22E221204600F027FE10BD773400081D
:1014B00010B5044602222321204600F01DFE04231D
:1014C0001E4A2A21204600F0D9FD04231B4A302160
:1014D000204600F0D3FD30222121204600F00CFEF2
:1014E00001222221204600F007FE3322252120463A
:1014F00000F002FE04222621204600F0FDFD0F220E
:101500002021204600F0F8FD09223121204600F07C
:10151000F3FD01223D21204600F0EEFD00223C219A
:10152000204600F0E9FD70222721204600F0E4FD6E
:10153000FF22E221204600F0DFFD10BD54340008F8
:1015400010B5044602222321204600F0D5FD0523D4
:101550001E4A2A21204600F091FD05231B4A302116
:10156000204600F08BFD3F222121204600F0C4FDE3
:1015700001222221204600F0BFFD12222521204613
:1015800000F0BAFD04222621204600F0B5FD0F220E
:101590002021204600F0B0FD0A223121204600F033
:1015A000ABFD01223D21204600F0A6FD00223C219A
:1015B000204600F0A1FD70222721204600F09CFD6E
:1015C000FF22E221204600F097FD10BD22340008E2
:1015D00010B5044602222321204600F08DFD05238C
:1015E0001E4A2A21204600F049FD05231B4A3021CE
:1015F000204600F043FD30222121204600F07CFDF2
:1016000001222221204600F077FD122225212046CA
:1016100000F072FD21222621204600F06DFD0F22F0
:101620002021204600F068FD0A223121204600F0EA
:1016300063FD00223D21204600F05EFD01223C2199
:10164000204600F059FD70222721204600F054FD6D
:10165000FF22E221204600F04FFD10BD13340008A8
:1016600010B5044601222321204600F045FD052344
:101670001E4A2A21204600F001FD05231B4A302185
:10168000204600F0FBFC30222121204600F034FDF2
:1016900001222221204600F02FFD1922252120467B
:1016A00000F02AFD04222621204600F025FD0F220D
:1016B0002021204600F020FD06223121204600F0A6
:1016C0001BFD01223D21204600F016FD00223C2199
:1016D000204600F011FD70222721204600F00CFD6D
:1016E000FF22E221204600F007FD10BD4034000833
:1016F00010B504461CB900202749086003E000200B
:1017000025490C31086001222321204600F0F4FC19
:101710000323224A2A21204600F0B0FC0323204A5A
:101720003021204600F0AAFC01222121204600F0B1
:10173000E3FC01222221204600F0DEFC2A222521A2
:10174000204600F0D9FC04222621204600F0D4FCDB
:101750000F222021204600F0CFFC06223D2120460A
:1017600000F0CAFC01223C21204600F0C5FC70229A
:101770002721204600F0C0FCFF22E221204600F095
:10178000BBFC1CB901200449086003E001200249A8
:101790000C31086010BD0000988121420934000816
:1017A0000434000870B504460D461CB900203A49BF
:1017B000086003E0002038490C310860152D60D224
:1017C000DFE805F00B0F13171B1F23272B2F3337D1
:1017D0003B3F43474B4F53575B002046FFF7F8FE14
:1017E0004FE0204600F09AFA4BE0204600F06EFBF6
:1017F00047E02046FFF7A4FE43E0204600F0FEF954
:101800003FE0204600F0DAF83BE02046FFF730FDED
:1018100037E0204600F0AAF933E0204600F0C6FA8F
:101820002FE02046FFF71CFF2BE0204600F036F8A3
:1018300027E0204600F02AFA23E0204600F076F860
:101840001FE02046FFF734FE1BE02046FFF708FFAD
:1018500017E02046FFF79CFD13E0204600F03EF91C
:101860000FE02046FFF74CFD0BE0204600F0EEF8BD
:1018700007E02046FFF7D4FD03E0204600F0DEFA43
:1018800000BF00BF1CB901200349086003E001202C
:1018900001490C31086070BD9881214210B50446A1
:1018A00002222321204600F027FC04231E4A2A217D
:1018B000204600F0E3FB04231B4A3021204600F0C1
:1018C000DDFB30222121204600F016FC01222221DE
:1018D000204600F011FC20222521204600F00CFCBF
:1018E00020222621204600F007FC0F22202120463E
:1018F00000F002FC08223121204600F0FDFB01220D
:101900003D21204600F0F8FB00223C21204600F05B
:10191000F3FB70222721204600F0EEFBFF22E2219C
:10192000204600F0E9FB10BD4534000810B5044620
:1019300002222321204600F0DFFB04231E4A2A2135
:10194000204600F09BFB04231B4A3021204600F078
:1019500095FB30222121204600F0CEFB01222221DE
:10196000204600F0C9FB12222521204600F0C4FBCE
:1019700024222621204600F0BFFB0F2220212046F2
:1019800000F0BAFB0A223121204600F0B5FB01220B
:101990003D21204600F0B0FB00223C21204600F013
:1019A000ABFB70222721204600F0A6FBFF22E2219C
:1019B000204600F0A1FB10BD4F34000810B50446CE
:1019C00002222321204600F097FB05231E4A2A21EC
:1019D000204600F053FB05231B4A3021204600F02F
:1019E0004DFB30222121204600F086FB01222221DE
:1019F000204600F081FB12222521204600F07CFBCE
:101A000024222621204600F077FB0F2220212046A9
:101A100000F072FB0A223121204600F06DFB01220A
:101A20003D21204600F068FB00223C21204600F0CA
:101A300063FB70222721204600F05EFBFF22E2219B
:101A4000204600F059FB10BD2C34000810B50446A8
:101A500002222321204600F04FFB04231E4A2A21A4
:101A6000204600F00BFB04231B4A3021204600F0E7
:101A700005FB30222121204600F03EFB01222221DD
:101A8000204600F039FB14222521204600F034FBCB
:101A900004222621204600F02FFB0F222021204681
:101AA00000F02AFB0A223121204600F025FB01220A
:101AB0003D21204600F020FB00223C21204600F082
:101AC0001BFB70222721204600F016FBFF22E2219B
:101AD000204600F011FB10BD6D34000810B504461F
:101AE00002222321204600F007FB04231E4A2A215C
:101AF000204600F0C3FA04231B4A3021204600F0A0
:101B0000BDFA30222121204600F0F6FA01222221DE
:101B1000204600F0F1FA12222521204600F0ECFACE
:101B200024222621204600F0E7FA0F222021204619
:101B300000F0E2FA08223121204600F0DDFA01220D
:101B40003D21204600F0D8FA00223C21204600F03A
:101B5000D3FA70222721204600F0CEFAFF22E2219C
:101B6000204600F0C9FA10BD6334000810B50446E1
:101B700001222321204600F0BFFA05231E4A2A2114
:101B8000204600F07BFA05231B4A3021204600F056
:101B900075FA30222121204600F0AEFA01222221DE
:101BA000204600F0A9FA10222521204600F0A4FAD0
:101BB00004222621204600F09FFA0F2220212046F1
:101BC00000F09AFA06223121204600F095FA01220F
:101BD0003D21204600F090FA00223C21204600F0F2
:101BE0008BFA70222721204600F086FAFF22E2219C
:101BF000204600F081FA10BD3634000810B50446C6
:101C000002222321204600F077FA05231E4A2A21CA
:101C1000204600F033FA05231B4A3021204600F00D
:101C20002DFA30222121204600F066FA01222221DD
:101C3000204600F061FA12222521204600F05CFACD
:101C400024222621204600F057FA0F222021204688
:101C500000F052FA08223121204600F04DFA01220C
:101C60003D21204600F048FA00223C21204600F0A9
:101C700043FA70222721204600F03EFAFF22E2219B
:101C8000204600F039FA10BD2734000810B504468C
:101C900002222321204600F02FFA04231E4A2A2183
:101CA000204600F0EBF904231B4A3021204600F0C7
:101CB000E5F930222121204600F01EFA01222221DE
:101CC000204600F019FA1C222521204600F014FAC3
:101CD00024222621204600F00FFA0F222021204640
:101CE00000F00AFA08223121204600F005FA01220C
:101CF0003D21204600F000FA00223C21204600F061
:101D0000FBF970222721204600F0F6F9FF22E2219C
:101D1000204600F0F1F910BD4A34000810B5044621
:101D200003222321204600F0E7F905231E4A2A2139
:101D3000204600F0A3F905231B4A3021204600F07D
:101D40009DF93F222121204600F0D6F93F22222191
:101D5000204600F0D1F928222521204600F0CCF9B8
:101D600004222621204600F0C7F90B22202120461C
:101D700000F0C2F90A223121204600F0BDF901220B
:101D80003D21204600F0B8F900223C21204600F019
:101D9000B3F970222721204600F0AEF9FF22E2219C
:101DA000204600F0A9F910BD1834000810B504460B
:101DB00001222321204600F09FF903231E4A2A21F5
:101DC000204600F05BF903231B4A3021204600F037
:101DD00055F930222121204600F08EF901222221DE
:101DE000204600F089F92A222521204600F084F9B6
:101DF00004222621204600F07FF90F2220212046D0
:101E000000F07AF907223121204600F075F900220E
:101E10003D21204600F070F901223C21204600F0CF
:101E20006BF970222721204600F066F9FF22E2219B
:101E3000204600F061F910BD3B34000810B504469F
:101E400001222321204600F057F903231E4A2A21AC
:101E5000204600F013F903231B4A3021204600F0EE
:101E60000DF930222121204600F046F901222221DD
:101E7000204600F041F932222521204600F03CF9AD
:101E800004222621204600F037F90F222021204687
:101E900000F032F910223121204600F02DF9012204
:101EA0003D21204600F028F900223C21204600F088
:101EB00023F970222721204600F01EF9FF22E2219B
:101EC000204600F019F910BD7C34000810B5044616
:101ED00003222321204600F00FF905231E4A2A2160
:101EE000204600F0CBF805231B4A3021204600F0A5
:101EF000C5F830222121204600F0FEF801222221DF
:101F0000204600F0F9F810222521204600F0F4F8D0
:101F100004222621204600F0EFF80F22202120463F
:101F200000F0EAF80A223121204600F0E5F801220B
:101F30003D21204600F0E0F800223C21204600F040
:101F4000DBF870222721204600F0D6F8FF22E2219C
:101F5000204600F0D1F810BD1D3400082DE9F047EF
:101F60008046894615461E46B8F1000F16D100205E
:101F7000174908604946404600F024FB0746002404
:101F800006E0FF21404600F01DFB2855601CC4B24E
:101F9000B442F6DB01200E49086015E000200D492F
:101FA00008604946404600F00DFB0746002406E065
:101FB000FF21404600F006FB2855601CC4B2B44225
:101FC000F6DB0120034908603846BDE8F0870000D1
:101FD00090012142B081214270B505460E4685B977
:101FE0000020114908603146284600F0EBFAFF2135
:101FF000284600F0E7FA044601200C49C1F8900198
:102000000FE000200A4908603146284600F0DAFA5D
:10201000FF21284600F0D6FA044601200549C1F800
:10202000B001204670BD0000900121420000214215
:10203000B08121420080214270B506460D46102134
:10204000304600F013FB07213046FFF7C5FF04467A
:1020500022462721304600F04FF804F0400050B1EE
:102060000A232A4661213046FFF778FFFF22E2214A
:10207000304600F041F8204670BD00002DE9F047E1
:102080008046894615461E46B8F1000F16D100203D
:10209000174908604946404600F094FA0746002474
:1020A00006E015F8011B404600F08CFA601CC4B233
:1020B000B442F6DB01200E49086015E000200D490E
:1020C00008604946404600F07DFA0746002406E0D5
:1020D00015F8011B404600F075FA601CC4B2B4420A
:1020E000F6DB0120034908603846BDE8F0870000B0
:1020F00090012142B08121422DE9F04104460E4673
:10210000154684B90020114908603146204600F088
:1021100059FA07462946204600F054FA01200C4996
:10212000C1F890010FE000200A49086031462046BE
:1021300000F048FA07462946204600F043FA0120FD
:102140000549C1F8B0013846BDE8F081900121424F
:1021500000002142B08121420080214208B54FF4A5
:10216000C06000F071F826208DF8000001208DF885
:10217000010002208DF8020001208DF8030068465E
:1021800000F02AF827208DF8000001208DF80100CA
:102190008DF802008DF80300684600F01DF8252038
:1021A0008DF8000000208DF8010001208DF802005C
:1021B0008DF80300684600F00FF81D208DF8000030
:1021C00000208DF801008DF8020001208DF8030039
:1021D000684600F001F808BD70B5002100230F2209
:1021E000C47804B3154C246804F4E064C4F5E064D6
:1021F000210AC1F10403CA40447804FA03F1847847
:102200001440214309010E4C0678A155047804F0CE
:102210001F050124AC4005786D11AD0005F1E025E6
:10222000C5F8004109E0047804F01F050124AC4022
:10223000044D0678761145F8264070BD0CED00E09F
:1022400000E400E080E100E002490143024A11603D
:10225000704700000000FA050CED00E07047000038
:1022600029B1064AD2690243044BDA6104E0034A09
:10227000D2698243014BDA617047000000100240CE
:1022800029B1064A92690243044B9A6104E0034A69
:1022900092698243014B9A6170470000001002402E
:1022A00070B5012144F20D00FFF7EAFF0121022081
:1022B000FFF7D6FF042000F013FB1249B1F1807F35
:1022C00000D31DE021F07F40401E4FF0E02250611E
:1022D00050170F22002807DA13071D0E0A4B00F0D3
:1022E0000F04241F1D5503E013071C0E074B1C543D
:1022F00000BF00204FF0E02290610720106100BF76
:1023000070BD000080A9030018ED00E000E400E0CB
:1023100070B5002100230024002200252C4E766891
:1023200006F00C0121B1042905D0082921D105E0CE
:10233000284E066020E0274E06601DE0244E766899
:1023400006F47013224E766806F48034022606EBFB
:1023500093431CB9204E5E43066009E01C4E76682C
:10236000C6F34046751C1B4EB6FBF5F65E43066091
:1023700002E0184E066000BF00BF154E766806F0FA
:10238000F0010909154E725C0668D6404660104E91
:10239000766806F4E061090A104E725C4668D64021
:1023A00086600B4E766806F46051C90A0B4E725C6B
:1023B0004668D640C660064E766806F44041890BF2
:1023C000074E725CC668B6FBF2F6066170BD00008F
:1023D0000010024000127A0000093D009000002029
:1023E000A000002010B586B00024142101A8FDF73C
:1023F000C2FE0A2201A9084800F012F800BF07E057
:1024000001A810F81400054A02F81400601CC4B2B8
:102410000A2CF5DB06B010BD0000030848050020BB
:1024200070B504460D461646002300BF07E020465F
:10243000FEF722FE25F81300A41C581CC3B2B342B9
:10244000F5DB70BD00B587B0012141F20500FFF753
:1024500017FFE020ADF8180018208DF81B000320AE
:102460008DF81A0006A91648FEF777FDE0211448FA
:10247000FEF700FE0020ADF804004FF48270ADF8C6
:1024800006000020ADF80800ADF80A00ADF80C0019
:102490004FF40070ADF80E001820ADF810000020C9
:1024A000ADF812000720ADF8140001A9054800F0AE
:1024B0006BF80121034800F04DF807B000BD0000A3
:1024C000000801400030014000B587B001218803B9
:1024D000FFF7C6FE01210920FFF7D2FE4FF460404E
:1024E000ADF8180018208DF81B0003208DF81A0095
:1024F00006A91648FEF731FD4FF460411348FEF778
:10250000B9FD0020ADF804004FF48270ADF806006C
:102510000020ADF80800ADF80A00ADF80C004FF44B
:102520000070ADF80E001820ADF810000020ADF8D6
:1025300012000720ADF8140001A9054800F024F8A6
:102540000121034800F006F807B000BD000C01406F
:102550000038004021B1028842F04002028004E0CD
:1025600002884FF6BF731A4002807047024600206F
:1025700013890B400BB1012000E000207047014699
:10258000888970478181704710B50022028802F463
:1025900041520B884C8823438C882343CC882343A7
:1025A0000C8923434C8923438C892343CC892343BF
:1025B0001A430280838B4FF2FF74234083830B8A7C
:1025C000038210BD2DE9F04106460F4626BB06E00A
:1025D000601CC4B2C82C02DB0020BDE8F0810221DF
:1025E0002048FFF7C3FF0028F2D039461D48FFF707
:1025F000C9FF002405E0601CC4B2C82C01DB002028
:10260000EBE701211748FFF7B1FF0028F3D0154889
:10261000FFF7B5FFC5B222E005E0601CC4B2C82CCC
:1026200001DB0020D9E702210F48FFF79FFF0028B8
:10263000F3D039460C48FFF7A5FF002405E0601CE5
:10264000C4B2C82C01DB0020C7E701210648FFF710
:102650008DFF0028F3D00448FFF791FFC5B228464C
:10266000BBE70000003001400038004070B505466F
:102670000C467DB90F4800884FF6C77108400D49D8
:102680000880084600882043088001210A48FFF797
:1026900061FF0EE0084800884FF6C7710840064900
:1026A0000880084600882043088001210248FFF77F
:1026B00051FF70BD0030014000380040704770B5D8
:1026C00004460D4629462046FEF708FC70BD000072
:1026D00010B586B00024142101A8FDF74CFD00BF01
:1026E00007E00B4830F8140001A921F81400601C21
:1026F000C4B20A2CF5DB074800F0EAF80A2201A967
:10270000044800F009F800F07AFC06B010BD0000A3
:1027100034050020000003082DE9F04105460F466E
:102720001646002400BF07E037F814102846FFF7CC
:10273000C6FFAD1C601CC4B2B442F5DBBDE8F0813D
:1027400070B504460D46034A2946204600F028F895
:1027500070BD00000038014010B504460249204613
:1027600000F00EF810BD00000044004010B5044613
:102770000249204600F02DF810BD00000044004042
:1027800070B504460D4600BF8021284600F064FB6A
:102790000028F9D02146284600F02BFC012070BD0E
:1027A0002DE9F04104460D46164614B90120BDE856
:1027B000F0810AE014F8017B31463846FFF7E0FF6C
:1027C00008B90020F3E7681E85B2002DF2D1012080
:1027D000EDE770B504460E460CB9012070BD11E05E
:1027E00014F8015B0A2D06D131460D20FFF7C8FF12
:1027F00008B90020F2E731462846FFF7C1FF08B9C3
:102800000020EBE720780028EAD10120E6E710B5A8
:1028100000F002F810BD00000CB5002001900090FF
:102820002A48006840F480302849086000BF2748E3
:10283000006800F4003000900198401C019000985E
:1028400018B90198B0F5A06FF1D12048006800F4E4
:10285000003010B10120009001E0002000900098AD
:10286000012831D119484068184948600846406835
:1028700048600846406848600846406820F47C107C
:1028800048600846406840F4981048600846006870
:1028900040F08070086000BF0C48006800F00070D5
:1028A0000028F9D00948406820F003000749486033
:1028B0000846406840F00200486000BF0348406896
:1028C00000F00C000828F9D10CBD000000100240F7
:1028D00010B50446FEF722FB2046FEF7B5FA10BD00
:1028E000042808D14FF0E021096941F004014FF0BC
:1028F000E022116107E04FF0E021096921F00401B5
:102900004FF0E022116170477047000010B5144885
:10291000006840F00100124908600846406811490B
:1029200008400F494860084600680F4908400C49B4
:1029300008600846006820F4802008600846406867
:1029400020F4FE0048604FF41F0088600020C86239
:10295000FFF75DFF4FF000600449086010BD000004
:10296000001002400000FFF8FFFFF6FE08ED00E057
:1029700010B50121204800F07EF800283AD001214E
:102980001D4800F069F81D480088401C1B4908805C
:102990001B480088401C1A4908801A480088401CBF
:1029A0001849088018480078C0B14FF400711748E2
:1029B000FEF760FB16480088401C15490880084651
:1029C0000088B0F5C87F09DB4FF400710F48FEF7AF
:1029D0004FFB00200E4908800B4908700948008809
:1029E00041F28831884202D1002006490880012046
:1029F0000849087010BD00000004004026000020B7
:102A00003A000020280000202C0000200010014087
:102A10002E0000202A0000203EB505460C4601216C
:102A20000220FFF71DFCADF80450ADF80040002077
:102A3000ADF80600ADF802006946064800F036F829
:102A400001221146034800F027F80121014800F057
:102A500006F83EBD00040040CA430282704721B11F
:102A6000028842F00102028004E002884FF6FE7301
:102A70001A400280704730B502460020002300242F
:102A8000158A05EA0103958905EA010413B10CB121
:102A9000012000E0002030BD1AB183890B438381FF
:102AA00002E083898B438381704700000022028803
:102AB0001D4B98420ED01D4B98420BD0B0F1804F69
:102AC00008D01B4B984205D01A4B984202D01A4BA3
:102AD000984204D14FF68F731A404B881A43174B14
:102AE000984207D0164B984204D04FF6FF431A4045
:102AF000CB881A4302808B8883850B8803850A4B19
:102B000098420BD0094B984208D00E4B984205D002
:102B10000D4B984202D00D4B984201D10B7A03869F
:102B20000123838270470000002C014000340140E3
:102B30000004004000080040000C0040001000406D
:102B400000140040004001400044014000480140A2
:102B500010B540F22551124800F08BF988B140F2CF
:102B600025510F4800F0CFF80D4800F03DFAC4B2EF
:102B70000C480D49097844540B480078401C0A4918
:102B800008700821064800F067F9012806D10821DD
:102B9000034800F0AFF8024800F026FA10BD00002C
:102BA000003801400C0100200300002010B540F265
:102BB0002551124800F05DF988B140F225510F48C7
:102BC00000F0A1F80D4800F00FFAC4B20C480D490E
:102BD000097844540B480078401C0A4908700821C1
:102BE000064800F039F9012806D10821034800F011
:102BF00081F8024800F0F8F910BD000000440040E0
:102C0000F40400208D00002010B586B00446012198
:102C10000520FFF735FB01214804FFF721FB0420C5
:102C2000ADF8140003208DF8160018208DF8170059
:102C300005A91548FEF791F90820ADF81400042005
:102C40008DF8170005A91048FEF787F901940020B8
:102C5000ADF80800ADF80A00ADF80C00ADF81000B2
:102C60000C20ADF80E0001A9084800F051F901222E
:102C700040F22551054800F026F90121034800F0F3
:102C800051F806B010BD00000008014000440040AB
:102C900010B540F22551144800F0EBF8B0B140F205
:102CA0002551114800F02FF80F4800F09DF9C4B2EB
:102CB0000E480F49097844540D480078401C0C49CF
:102CC00008700846007800F00F00087008210648D8
:102CD00000F0C2F8012806D10821034800F00AF8E4
:102CE000014800F081F910BD00480040D4010020E7
:102CF0000900002001F40072B2F5007F00D100BF8E
:102D0000CA430280704710B50022002340F66A14BF
:102D1000A14200D100BF0A1201249440A3B2DC43B7
:102D2000048010BD21B1828942F40052828104E006
:102D300082894DF6FF731A408281704700B585B0D5
:102D4000012144F20400FFF79BFA4FF40070ADF844
:102D5000000003208DF8020018208DF8030069465A
:102D60003948FEF7FAF84FF48060ADF8000004200F
:102D70008DF8030069463448FEF7EFF84FF416402B
:102D800001900020ADF80800ADF80A00ADF80C0085
:102D9000ADF810000C20ADF80E0001A92B4800F092
:102DA000B7F8012240F22551284800F08CF80121A3
:102DB0002648FFF7B7FF01218804FFF751FA0121E8
:102DC0000820FFF75DFA4FF48060ADF800000320A3
:102DD0008DF8020018208DF8030069461C48FEF7A4
:102DE000BCF84FF40060ADF8000004208DF803003B
:102DF00069461748FEF7B1F84FF49650019000204D
:102E0000ADF80800ADF80A00ADF80C00ADF8100000
:102E10000C20ADF80E0001A90E4800F079F801A9C8
:102E20000C4800F075F8012240F22551094800F0E5
:102E30004AF801210748FFF775FF40210348FFF7D3
:102E400059FF05B000BD00000008014000380140F6
:102E5000000C01400048004002460020B1F5007F10
:102E600000D100BF13880B400BB1012000E000200F
:102E7000704770B50246002400230025002040F66C
:102E80006A16B14200D100BFC1F3421501F01F0321
:102E9000012606FA03F3012D02D19689334006E09C
:102EA000022D02D1168A334001E0968A33400C127B
:102EB000012606FA04F41688344013B10CB101203F
:102EC00000E0002070BDF0B5034600240026002578
:102ED000002040F66A17B94200D100BF1846C1F37E
:102EE000421401F01F06012707FA06F5012C01D153
:102EF0000C3004E0022C01D1103000E014301AB183
:102F000007682F43076002E00768AF430760F0BD22
:102F10002DE9F04786B005460E460024A24600BFC4
:102F2000A1460027B08900B100BF2F462C8A4CF67D
:102F3000FF700440F08804432C82AC894EF6F310F5
:102F40000440B08831890843718908430443AC8147
:102F5000AC8A4FF6FF400440B0890443AC8201A81C
:102F6000FFF7D6F91F48874202D1DDF810A001E033
:102F7000DDF80CA0A88900F4004040B10AEBCA00BB
:102F800000EB0A1031684900B0FBF1F807E00AEBEA
:102F9000CA0000EB0A1031688900B0FBF1F8642028
:102FA000B8FBF0F004012009642101FB1089A88915
:102FB00000F4004040B1322000EBC900B0FBF1F05A
:102FC00000F00700044308E0322000EB0910642100
:102FD000B0FBF1F000F00F0004432C8106B0BDE817
:102FE000F08700000038014001468888C0F30800DF
:102FF0007047C1F308028280704700BFFEE710B53A
:10300000FDF762FF10BD0000014A024900F013B84D
:1030100085300008A400002002E008C8121F08C183
:10302000002AFAD170477047002001E001C1121F49
:10303000002AFBD170472DE9F04116460F460446A1
:10304000002503E03946B047641C6D1C2078002839
:10305000F8D12846BDE8F08110B502460BE0C82043
:1030600007E0122101E04B1E99B20029FBDC431E50
:1030700098B20028F5DC131EA2F10104A2B2EED131
:1030800010BD000070B504460D46E0B20549088049
:1030900000BF40210348001FFFF7DEFE0028F8D0E4
:1030A000204670BD0438014008B501211020FFF70B
:1030B000E7F80120ADF8000010208DF80300032090
:1030C0008DF8020069460D48FDF747FF01210B48C6
:1030D000FDF7D0FF4FF40070ADF8000010208DF820
:1030E000030003208DF8020069460448FDF735FF10
:1030F0004FF400710148FDF7BBFF08BD001001400F
:10310000FFF7CEF8FFF72AF840F271210420FDF70F
:10311000D5FFFDF7CFFF41F61F410920FFF77CFCEB
:10312000FFF7C2FFFFF70AFE4FF4E130FFF76CFD37
:10313000FEF720F8FDF7BEFF02E051A0FFF764FFA5
:103140000120FDF7EBFF0028F7D1FDF7C1FDFDF7EA
:10315000B1FF4F480068C0434E49C1F88001C82004
:10316000FFF77AFF4B48D0F88001C0434949C1F8C6
:103170008001062148A0FDF74CFE49A0FFF7F6FAB2
:10318000FDF798FF47A0FFF73FFF0120FEF7B0FAD9
:10319000FFF728F94C4800784C4908700846007839
:1031A000152860D2DFE800F00B0F13171B1F232731
:1031B0002B2F33373B3F43474B4F53575B0044A0C4
:1031C000FFF722FF4FE045A0FFF71EFF4BE046A0B0
:1031D000FFF71AFF47E047A0FFF716FF43E048A0BC
:1031E000FFF712FF3FE049A0FFF70EFF3BE04BA0C7
:1031F000FFF70AFF37E04CA0FFF706FF33E04EA0D1
:10320000FFF702FF2FE04FA0FFF7FEFE2BE050A0DC
:10321000FFF7FAFE27E051A0FFF7F6FE23E053A0E8
:10322000FFF7F2FE1FE056A0FFF7EEFE1BE058A0EE
:10323000FFF7EAFE17E05AA0FFF7E6FE13E05CA0F6
:10324000FFF7E2FE0FE05EA0FFF7DEFE0BE060A0FE
:10325000FFF7DAFE07E062A0FFF7D6FE03E064A006
:10326000FFF7D2FE00BF00BF012065490870322081
:10327000FFF7F2FE03E0FCF7AFFFFDF717FAFAE7FE
:1032800054686520322E3447204572726F722100D7
:1032900080012242000022423132333435360000B0
:1032A0000A0000000A5043B6D4C2EBC8EDBCFECD04
:1032B000A8D3C3B0E6B1BE56322E342D32303139E8
:1032C000303930360A000000480500203200002066
:1032D000BDADCEF7D0ADD2E90D0A0000CCECB2A85E
:1032E000D0ADD2E90D0A0000D4C6C4CFD0ADD2E92A
:1032F0000D0A0000B9F3D6DDD0ADD2E90D0A000009
:10330000CBC4B4A8D0ADD2E90D0A0000C4DAC3C959
:10331000B9C5D0ADD2E90D0A00000000B0B2BBD5EE
:10332000D0ADD2E90D0A0000C9BDCEF7F6CEC5B5C5
:10333000D0ADD2E90D0A000056434F4DB2E2CAD4D7
:103340000D0A0000C1C9C4FEB5E7D0C50D0A0000D2
:10335000C1C9C4FED2C6B6AF0D0A00005470D7A8CA
:10336000D3C3D0ADD2E90D0A00000000C4DAC3C94E
:10337000B9C5D2C6B6AFD0ADD2E90D0A0000000083
:10338000B9E3CEF7D2C6B6AFD0ADD2E90D0A000090
:10339000CBC4B4A8B5E7D0C5D0ADD2E90D0A0000C2
:1033A000B8A3BDA8D5E6D7C6D0ADD2E90D0A0000B6
:1033B000CBD5D6DDC4BEC0BCD0ADD2E90D0A00006D
:1033C000D6D8C7ECD2C6B6AFD0ADD2E90D0A000050
:1033D000C9BDCEF7D2C6B6AFD0ADD2E90D0A000056
:1033E000B8CACBE0D2C6B6AFD0ADD2E90D0A000064
:1033F000D0C5B4EFB7E1D0ADD2E90D0A00000000AE
:103400002B000020344310100134431010013320EE
:103410000D547933200D54793443101001011010EC
:1034200043343223ABBA013412BBAA01341286757D
:10343000014656431000346E46100134431010010B
:10344000862C95010136E4A7BC014218BAE8013484
:103450001286750133200D5400862C9500005A45C4
:103460004E4B00AABB1234003412BBAA00254310F5
:103470001200E77EE300004222B6E900C013E30039
:1034800000000000A434000800000020A800000094
:10349000183000084C350008A8000020585F0000D4
:1034A00028300008000000000000000000000000BC
:1034B000D1D1E0D000000000D2D200000000000016
:1034C00000000000000000000000000000000000FC
:1034D00000000000000000000000000000000000EC
:1034E0000000000000000000000000000000313279
:1034F0003334353637383931323334353637383975
:103500000000000000000000000000000000313258
:103510003334353637383931323334353637383954
:10352000000000000000000000000000000000009B
:103530000000000000000000010203040102030477
:0C3540000607080902040608000000004D
:0400000508000131BD
:00000001FF
